:100000000C9473060C9490060C9490060C94900635
:100010000C9490060C9490060C9490060C94900608
:100020000C9490060C9490060C940E2B0C94E02BE0
:100030000C94F7240C9490060C9490060C94900663
:100040000C9490060C9490060C9490060C949006D8
:100050000C9490060C9480250C9490060C949006B9
:100060000C9490060C9490060C9490060C949006B8
:100070000C9490060C9490060C9490060C949006A8
:100080000C9490060C9490060C9490060C94900698
:100090000C9490060C9490060C9490060C94900688
:1000A0000C9490060C9490060C949006CD0ACD0A00
:1000B000F90AF90A670B850B660C660C8A0BF20BC2
:1000C000030C030C8F1B921BBC1BCF1BD71BE21B0B
:1000D000E51BE51BE51B2D1C2D1CEA1BED1BF21B74
:1000E000FF1B0C1C0F1C131C201C8E1C001D961CBF
:1000F000601C641C9A1C671C9D1CA81C721CF61CAE
:10010000761CAC1C7A1CB01CDA1C7E1CB41CE41CD3
:10011000841CBA1CC41C6B1CA11C6E1CA41C891C56
:10012000BF1CD01CF01CF21C5C1C921C091D772308
:100130007D236B237123832389238F23482C6F2CEA
:10014000672D6F2C672DBB2CDE2C672D352D442D94
:10015000415254005500560001000000000000000C
:1001600000000000000000000000000000005F0030
:100170006000610057000100000000000000000066
:100180000000000000000000000000005C005D00B6
:100190005E005700010000000000000000000000A9
:1001A0000000000000000000000059005A005B0041
:1001B00058000100000000000000000000000000E6
:1001C00000000000000000006200620063005800B0
:1001D000010000000000000000000000000000001E
:1001E00000000000000001001E001F002000210090
:1001F0002200230024002500260027000100010022
:1002000001000100290014001A0008001500170061
:100210001C0018000C00120013002A005F00600090
:1002200061002B0004001600070009000A000B0003
:100230000D000E000F00330034005C005D005E0016
:10024000E1001D001B000600190005001100100050
:10025000360037003800282259005A005B00E000C1
:10026000E300E200E2002252E1002C002352E7000A
:10027000E6004C00E400620062006300010001003F
:100280000100010001000100010001000100010066
:100290000100010001000100010001003A003B00E3
:1002A0003C003D003E003F00400041004200430052
:1002B000530054005500560035001E001F0020005A
:1002C0002100220023002400250026002700010031
:1002D0000100010057000100440045000100010039
:1002E00001002800E500E70037242A210100010071
:1002F000010058000100010001000100010001009F
:100300002800E500010001000100010001000100DA
:1003100001000100010001000100010001000100D5
:1003200001000100010001000100010001000100C5
:10033000007C2B00520001004900E000E1004B006E
:100340004A002D002E004C00010001000100390080
:10035000500051004F004600E100E0004E004D000B
:100360002F003000310001000100010001004800B1
:10037000010001000100010001000100E700E600AA
:1003800001000100010001000100405201000100D4
:100390000100010001000100010001000100010055
:1003A000010001000100010044454255473A206424
:1003B000697361626C65642E0A0044454255473A90
:1003C00020656E61626C65642E0A000A0025303279
:1003D00058006C65645F7461736B3A20004F6E6502
:1003E00073686F743A206163746976653A20256496
:1003F0000A000A002530313662003A2000253032EA
:1004000058000A722F632030313233343536373892
:10041000394142434445460A00290A002575002F08
:10042000002575005D28002564002000256400205B
:100430000025640020002564007C0025303258002F
:100440006D6F7573656B6579205B62746E7C782067
:1004500079207620685D287265702F61636C293A77
:10046000205B0000000000000000002A2B28000094
:100470000000000000000000000000000000290053
:100480000000002C1E3420212224342627252E365D
:100490002D3738271E1F20212223242526333336CB
:1004A0002E37381F0405060708090A0B0C0D0E0F1E
:1004B000101112131415161718191A1B1C1D2F31A1
:1004C00030232D350405060708090A0B0C0D0E0F05
:1004D000101112131415161718191A1B1C1D2F3181
:1004E00030354C000000000000000000000000005B
:1004F00000000000000000000000000000000000FC
:10050000000000000000007E0F00D4FFFFFFC700C6
:10051000000078313A0964656C6179282A31306DC0
:1005200073293A2025750A323A09696E7465727624
:10053000616C286D73293A2025750A333A096D617B
:10054000785F73706565643A2025750A343A0974DA
:10055000696D655F746F5F6D61783A2025750A3546
:100560003A09776865656C5F6D61785F7370656582
:10057000643A2025750A363A09776865656C5F74B8
:10058000696D655F746F5F6D61783A2025750A004B
:10059000703A097072696E742076616C7565730AC1
:1005A000643A097365742064656661756C74730AD6
:1005B00075703A092B310A646E3A092D310A6C7450
:1005C0003A092B31300A72743A092D31300A4553F9
:1005D000432F713A09717569740A0A73706565640D
:1005E000203D2064656C7461202A206D61785F7302
:1005F00070656564202A2028726570656174202FFB
:100600002074696D655F746F5F6D6178290A776822
:100610006572652064656C74613A20637572736FEE
:10062000723D25642C20776865656C3D25640A530E
:10063000656520687474703A2F2F656E2E77696B2C
:100640006970656469612E6F72672F77696B692FB6
:100650004D6F7573655F6B6579730A004D3E2000C1
:100660004D25753A25733E20003F0A003D20257533
:100670000A003F0A0064656661756C74730A0025A0
:10068000750A003F0A000A092D2056616C756573D2
:10069000202D0A00710A000A092D204D6F7573651F
:1006A0006B6579202D0A003F00433E20004C2564F5
:1006B0000A000A092D20537461747573202D0A688D
:1006C0006F73745F6B6579626F6172645F6C656490
:1006D0007328293A20253032580A6B6579626F6198
:1006E00072645F70726F746F636F6C3A2025303282
:1006F000580A6B6579626F6172645F69646C653A10
:1007000020253032580A74696D65725F72656164C4
:10071000333228293A202530386C580A00257300D6
:100720000A092D20436F6E736F6C65202D0A4553A7
:10073000432F713A09717569740A6D3A096D6F75C5
:1007400073656B65790A000A092D204D616769633D
:10075000202D0A443A094465627567204D6573731C
:1007600061676520546F67676C650A583A094D6187
:1007700074726978204465627567204D6F646520E6
:10078000546F67676C65202D2053686F77206B6509
:10079000797072657373657320696E206D61747210
:1007A000697820677269640A4B3A094B6579626F10
:1007B00061726420446562756720546F67676C6579
:1007C000202D2053686F77206B6579707265737385
:1007D000207265706F72740A4D3A094465627567DC
:1007E000204D6F75736520546F67676C650A563AC4
:1007F0000956657273696F6E0A533A0953746174CE
:1008000075730A433A0941637469766174652043DC
:100810006F6E736F6C65204D6F64650A46312D46AF
:1008200031303A0953776974636820746F204C61E2
:1008300079657220302D392028463130203D204CFA
:1008400030290A302D393A09537769746368207466
:100850006F204C6179657220302D390A475241561C
:10086000453A0953776974636820746F204C617945
:10087000657220302028616C7465726E6174652920
:100880000A423A094A756D7020746F20426F6F7486
:100890006C6F616465720A4553433A094A756D701D
:1008A00020746F20426F6F746C6F616465722028D2
:1008B000616C7465726E617465290A453A095072FB
:1008C000696E7420454550524F4D205365747469CC
:1008D0006E67730A4241434B53504143453A0943C3
:1008E0006C65617220454550524F4D0A006B657929
:1008F0006D61705F636F6E6669672E7261773A2013
:10090000253032580A2E737761705F636F6E747290
:100910006F6C5F636170736C6F636B3A2025750A4F
:100920002E636170736C6F636B5F746F5F636F6E68
:1009300074726F6C3A2025750A2E737761705F6C44
:1009400063746C5F6C6775693A2025750A2E73773E
:1009500061705F7263746C5F726775693A202575A8
:100960000A2E737761705F6C616C745F6C67756978
:100970003A2025750A2E737761705F72616C745F1F
:10098000726775693A2025750A2E6E6F5F67756903
:100990003A2025750A2E737761705F6772617665FC
:1009A0005F6573633A2025750A2E737761705F6205
:1009B00061636B736C6173685F6261636B737061B9
:1009C00063653A2025750A2E6E6B726F3A20257585
:1009D0000A2E737761705F6573636170655F636131
:1009E00070736C6F636B3A2025750A0064656275DD
:1009F000675F636F6E6669672E7261773A20253094
:100A000032580A2E656E61626C653A2025750A2E91
:100A10006D61747269783A2025750A2E6B6579626A
:100A20006F6172643A2025750A2E6D6F7573653A91
:100A30002025750A006565636F6E6669673A0A640A
:100A4000656661756C745F6C617965723A202575B5
:100A50000A003F000A6D6F7573653A206F66660A7B
:100A6000000A6D6F7573653A206F6E0A000A6B6538
:100A700079626F6172643A206F66660A000A6B657C
:100A800079626F6172643A206F6E0A000A6D617458
:100A90007269783A206F66660A000A6D617472693D
:100AA000783A206F6E0A000A64656275673A206FB3
:100AB00066660A000A64656275673A206F6E0A000E
:100AC0000A0A4A756D70696E6720746F20626F6FD5
:100AD000746C6F616465722E2E2E2000433E2000E0
:100AE000436C656172696E6720454550524F4D0AEF
:100AF000000A002530325820006B6579626F617200
:100B0000645F7265706F72743A20005B735D005BA6
:100B1000575D005B535D005B525D005B445D005BB5
:100B2000435D002203540068006500200035007812
:100B300000350020004B006500790062006F006105
:100B4000007200640000000C03640069003000695A
:100B500000620000000403090409027B0004010094
:100B6000A0FA09040000010301010009211101009C
:100B70000122400007058103080001090401000269
:100B80000300000009211101000122220007058253
:100B900003200001070503032000010904020001EE
:100BA00003000000092111010001227B00070584D8
:100BB00003200001090403000203000000092111C1
:100BC0000100012222000705850320000107050519
:100BD0000320000112010002000000082540B505B5
:100BE0000001010200010631FF0974A10109751518
:100BF0000026FF009520750881020976150026FF62
:100C000000952075089102C00660FF0961A10109E5
:100C100062150026FF009520750881020963150002
:100C200026FF00952075089102C005010902A10167
:100C300085020901A10005091901290815002501EE
:100C40009508750181020501093009311581257F5B
:100C500095027508810609381581257F950175086B
:100C60008106050C0A38021581257F9501750881DA
:100C700006C0C005010980A101850319012AB7003A
:100C8000150126B700950175108100C0050C0901FA
:100C9000A101850419012AA002150126A0029501CF
:100CA00075108100C005010906A101050719E02999
:100CB000E7150025019508750181029501750881E8
:100CC000010507190029FF150026FF009506750884
:100CD0008100050819012905950575019102950105
:100CE00075039101C00011241FBECFEFDAE0DEBF13
:100CF000CDBF12E0A0E0B1E0ECECFCE502C0059055
:100D00000D92A83CB107D9F723E0A8ECB2E001C0EE
:100D10001D92A73AB207E1F70E94AF170C94642E18
:100D20000C940000FF93EF93E091C802F091C90288
:100D3000309709F00995EF91FF910895FC01859195
:100D4000803011F0EFDFFBCF0895FF27E0E230E2C3
:100D500047FF0CC0419597FF09C0EDE26095709583
:100D600080959095611D711D811D911D27FF02C009
:100D7000219530E350E2AA27660F771F881F991F3D
:100D8000AA1FA41710F0A41B63955A95A9F7AA30BF
:100D900008F0A95FA05DAF93F3956115710581051A
:100DA000910541F7ED3211F4EF93F395F21718F432
:100DB0003F93F395FBCF8F91B5DFFA95E1F7089557
:100DC000E991F9918591803021F0853219F0AADFFF
:100DD000F9CF089520E0E89455915532C1F350338E
:100DE00011F4689455915A3348F4505390F3220FFC
:100DF000022E220F220F200D250FF4CF0EF4219585
:100E000089919991533619F3533729F1533559F193
:100E1000BC0188279927E8945C3621F4899199913F
:100E200068945591543639F446EF7EF077FF0DC043
:100E30008FEF9FEF0AC055374AE039F0583540E14F
:100E400021F0523642E009F00895FF93EF937DDFE1
:100E5000EF91FF91B7CFFF93EF93FC018191803029
:100E6000B9F360DFFBCFFF93EF9368DFF1CFDF9340
:100E7000CF93CDB7DEB72596A3DFCF91DF9108954D
:100E800084E008958430B0F46530A0F44F3090F4DD
:100E90009BE4899FF00111248FE0689FE00DF11D14
:100EA0001124E40FF11DEE0FFF1FE05BFE4F859153
:100EB0009491089580E090E0089581E0089581E0A4
:100EC00008950E945F07089508950E946407089599
:100ED000A5E0B0E0EEE6F7E00C94D02D49835A830C
:100EE0003091CF0289819A81311114C0662359F063
:100EF000222349F00E94200E182F682F89819A81A1
:100F00000E94FC0D03C00E940E0E182F69817A8189
:100F1000812F04C00E94200E69817A810E94F11401
:100F20002596E3E00C94EC2DFC01262F40815181A5
:100F30006281738184810E946807089581E0089529
:100F4000CF93DF93EC0160E00E949407BE010E9402
:100F50006507DF91CF910895E1E0F0E0DF0102C085
:100F6000AA0FBB1F6A95E2F7BD01DF0102C0AA0FFD
:100F7000BB1F4A95E2F7AD01462B01C0EE0F2A9543
:100F8000EAF7942F9823491302C08E2B0895E09519
:100F90008E230895242F462F682F8091EE020E9401
:100FA000AC070E945D0D08950E94731608950E947B
:100FB0006D16089508950E94E90C0E94DA072FEF3C
:100FC00084E39CE0215080409040E1F700C00000A5
:100FD00008950E94DB070E94A62508950E94DB0762
:100FE0000E94B72508950F931F93CF93DF938C0131
:100FF00061E00E949407EC01B8010E94351B882330
:1010000059F1B801CE010E946107882329F1B80186
:10101000CE010E945F238823F9F0B801CE010E941F
:10102000381C8823C9F0B801CE010E94C52288234C
:1010300099F0F80182818823F1F1C3308CE7D80759
:1010400081F160F4C130FCE7DF0769F1A8F4C11554
:10105000DC4789F50E94E907C0E031C0CB35FCE7E9
:10106000DF0739F1CC358CE7D80701F1CA35DC4709
:1010700011F50E946A121FC080915003C82FC095BD
:10108000C170C0FB80F980935003CC2329F08AEB18
:1010900093E00E949E06E0CF88EA93E00E949E06BD
:1010A0000EC00E9472120E94EE07D6CF0E946012FC
:1010B00002C00E946E12C8010E945D07C82F8C2FCB
:1010C000DF91CF911F910F9108950E94CF240E942C
:1010D000B40808950E94B8080E94D8240895829503
:1010E000982F937344E0949F900111248C7C8695F3
:1010F0008695282B822F8575880F2A7A2695822B34
:101100000895CF93DF93D92F0E946F08C82F8D2F9A
:101110000E946F082C2F30E0322F2227A901482B84
:10112000CA01DF91CF91089508950E94940808950F
:1011300081E008950895CF93DF93D82F0E949808F7
:10114000C82F882319F08D2F0E949A088C2FDF91C9
:10115000CF9108950895CF93C82F0E9495088C2FA2
:101160000E949B08CF91089580E00E94AB080895EB
:101170000E94AC230E94AB080895CF930E94AC2339
:10118000C82F8091CA02C81789F1C093CA020E9471
:1011900065256093CB027093CC028093CD0290932F
:1011A000CE028091500382FF1EC080FF04C082EDFA
:1011B00093E00E949E068091500380FF0CC01F9216
:1011C000CF938DEC93E09F938F930E9437070F90FE
:1011D0000F900F900F908091500380FF04C08BEC14
:1011E00093E00E949E068C2F0E94AB08CF91089539
:1011F000ABE0B0E0EEEFF8E00C94D12D4F835887D0
:1012000069877A878B8761110E9494119E012F5FF5
:101210003F4F86E0F90111928A95E9F785E0FE01DA
:101220003796D90101900D928A95E1F789819A81CB
:101230004C815D81452B31F09F3F31F491E08F3F30
:1012400019F403C091E001C090E090FF09C049810A
:101250005A816B817C818D819E810E94C01005C066
:10126000C9010E949E078111F2CF2B96E2E00C94F7
:10127000ED2DFC01808191810E944D0E0895662321
:1012800019F00E94341802C00E948F180E9406199B
:101290000895CF93882309F4A9C0C82F8238C1F4D8
:1012A0000E94AC2381FDA2C069E38091000190916E
:1012B00001010E9494240E94B8112FEF87EE93E061
:1012C000215080409040E1F700C0000069E319C060
:1012D000833801F50E94AC2380FD88C063E58091CE
:1012E0000001909101010E9494240E94B8112FEFF7
:1012F00081EE94E0215080409040E1F700C0000072
:1013000063E580910001909101010E9497240E9461
:10131000B8116CC08438C1F40E94AC2382FD66C051
:1013200067E480910001909101010E9494240E9441
:10133000B8112FEF81EE94E0215080409040E1F70A
:1013400000C0000067E4DDCF8CEF8C0F813AF8F429
:101350008C2F0E94CA20811149C06C2F80910001FE
:10136000909101010E945E24882349F06C2F8091A6
:101370000001909101010E9497240E94B8116C2FE6
:1013800080910001909101010E949424C0CF80E2DD
:101390008C0F883048F4C77081E001C0880FCA956F
:1013A000EAF70E947711B3CFEBE5EC0FE33040F49E
:1013B000F0E0EB5BFE4F808190E00E94082416C0B5
:1013C000E8E5EC0FE93150F4F0E0EE0FFF1FED5EC1
:1013D000FE4F808191810E942D2408C083E38C0FF1
:1013E000833120F461E08C2F0E943F09CF91089552
:1013F000882309F468C0823879F40E94AC2381FF05
:1014000062C069E380910001909101010E949424DF
:101410000E94B81169E310C08338B9F40E94AC236C
:1014200080FF51C063E580910001909101010E940D
:1014300094240E94B81163E580910001909101010C
:101440000E9497240E94B8110895843879F40E946C
:10145000AC2382FF38C067E48091000190910101C4
:101460000E9494240E94B81167E4E6CF9CEF980F85
:10147000913A10F4682FE0CF90E2980F983050F432
:10148000877091E001C0990F8A95EAF7892F0E9431
:101490007D11D8CF9BE5980F933028F480E090E041
:1014A0000E940824089598E5980F993128F480E067
:1014B00090E00E942D24089593E3980F933118F43F
:1014C00060E00E943F0908951F93CF93DF93182F88
:1014D000EB010E944909209741F08FE99FE00197B5
:1014E000F1F700C000002197F6CF812F0E94F80984
:1014F000DF91CF911F910895893319F060E070E07A
:1015000002C060E570E00E94640A0895882321F01B
:101510000E9477110E94B8110895882321F00E943B
:101520007D110E94B8110895A0E0B0E0EAE9FAE068
:101530000C94CB2D7C01162FC72FFC01D281058185
:1015400002950F700E946D118823B9F0DD23A9F078
:101550008C2F807F803421F080E2810F883068F00A
:101560008091810382FF09C082E00E941A120E94CA
:101570006D1191E0D82ED92601C0D12CCC2EC29469
:101580008FE0C8228C2D90E08C30910508F09EC130
:10159000FC01EA5AFF4F0C94B42D8C2F807FCF7042
:1015A000882311F0C295C07FDD2399F0CC2309F484
:1015B00079C180E2810F883010F0111104C08C2FA6
:1015C0000E94771103C08C2F0E9487110E94B811CE
:1015D00069C1812F0E94F809CC2309F477C180E208
:1015E000810F883038F1112329F18C2F0E948D1141
:1015F00024C08C2F807FCF70803211F0C295C07FC5
:10160000112319F01130D1F143C08091810382FD83
:1016100017C0DD2349F0CC2329F08C2F0E947711CD
:101620000E94B81180E03FC180E00E94F809CC23FD
:1016300009F44CC18C2F0E947D110E94B81146C143
:10164000DD2371F0002341F0013031F40E94971145
:101650008C2B0E94A1113AC10E9497118C2B23C0A0
:10166000011103C00E94AE112EC0013009F42EC139
:101670008C2F0E948D0A0E94AE1128C1DD2321F01B
:10168000063008F023C10EC0053008F01FC11BC092
:10169000DD2361F0002331F0F701858180FF02C175
:1016A0008F7085838C2F0E94860A10C1002359F009
:1016B000193309F008C1FFEF27EE83E0F150204015
:1016C0008040E1F7FEC08C2F0E948D0AFFC08C2F56
:1016D00086958695837019F0813061F0F7C0DD231F
:1016E00021F0812F9C2F937002C080E090E00E9437
:1016F0000824F4C0DD2321F0812F9C2F937002C0B9
:1017000080E090E00E942D24E9C06D2F812F0E947F
:101710003F09E4C08C2F837079F5D111DBC0412FD4
:10172000429546954770440F440F212F2F70042E89
:1017300001C0220F0A94EAF714FF08C08FE090E07E
:1017400001C0880F4A95EAF7809501C080E0C695F0
:10175000C695C370822BC23049F058F4C13019F0DD
:101760000E944E0DB7C00E94480DB4C00E94540D97
:10177000B1C00E94450DAEC0DD2319F08C2F8170E1
:1017800001C08695882309F4A5C0412F429546954E
:101790004770440F440F212F2F70042E01C0220FD9
:1017A0000A94EAF714FF08C08FE090E001C0880FA8
:1017B0004A95EAF7809501C080E0C695C695C3704A
:1017C000822BC23049F058F4C13019F00E949A0DB2
:1017D00081C00E94940D7EC00E94A00D7BC00E941B
:1017E0005D0D78C0CF70DD2339F08C2F0E946F0D16
:1017F000812F0E94860A6EC0812F0E948D0A8C2F35
:101800000E947B0D67C0123F21F128F4103F41F088
:10181000113FC1F043C0133F19F1143F79F03EC0AE
:10182000DD2341F0053008F051C08C2F8F710E94EC
:10183000880D4CC0063008F049C0F7CF8091810375
:1018400082FD18C0DD2339F08C2F8F710E946F0D3F
:101850003DC0DD23C9F38C2F8F710E947B0D36C0F4
:10186000DD2329F08C2F8F710E94660D2FC00E94FE
:10187000620D2CC0DD2349F0CF718C2F0E946F0DBB
:1018800063E08C2F0E94FC1121C081E00E941A129B
:101890000230E0F082E00E941A1218C0DD2331F01D
:1018A000002391F2812F0E94490910C0002399F270
:1018B000193349F49FEFE7EEF3E09150E040F04038
:1018C000E1F700C00000812F0E94F80988EF8C0D1D
:1018D000843020F40E94AC230E94AB08DD2089F004
:1018E0000E94691180FD0DC0F70112820E946311F0
:1018F0000E946F0DC7010E949E0C0E9463110E94FE
:101900007B0DCDB7DEB7E8E00C94E72D0F931F9366
:10191000CF93DF93EC01688179818A810E94580E10
:101920008C010E94A60D0E94380DB801CE010E94C4
:10193000940ADF91CF911F910F910895CF93DF9378
:10194000EC01988189812B813C81232B31F08F3FE1
:1019500031F481E09F3F19F403C081E001C080E0D1
:1019600080FD1AC0CE010E94F30781110FC00E94B2
:101970006D11882389F08A81882371F08091810319
:1019800082FF0AC082E00E941A1206C0CE010E94A5
:10199000860CCE010E94A007DF91CF91089580E0D0
:1019A00090E00E94082480E090E00E942D240E9494
:1019B00094110E94B8110E94A7190E940619089557
:1019C00080910001909101010E949A240E94CF0C05
:1019D00008950E9484110E94E00C089592959F70D2
:1019E000963079F010F4925001C09A50923068F419
:1019F000803F69F018F4883E40F409C0843F29F420
:101A000006C0883E20F0813F11F080E0089581E01B
:101A10000895FC019081818123813481232B31F051
:101A20008F3F31F481E09F3F19F403C081E001C092
:101A300080E080FD07C0808191810E944D0E0E9450
:101A4000EE0C089580E00895A5E0B0E0EAE2FDE044
:101A50000C94D12D2596E2E00C94ED2DA6E0B0E09B
:101A6000E4E3FDE00C94D12D2696E2E00C94ED2DFC
:101A7000089508950E94390D08950E943A0D089521
:101A80000E943D0D8093EF0208950E94400D08953D
:101A90009091EF02892B0E94400D08959091EF02E2
:101AA00089230E94400D08959091EF0289270E949A
:101AB000400D08950E94390D08950E945A0D80939B
:101AC000EE02089580E00E945D0D089591E001C04E
:101AD000990F8A95EAF7892F0E945D0D089521E0FC
:101AE00030E001C0220F8A95EAF78091EE02822B46
:101AF0000E945D0D089521E030E001C0220F8A951B
:101B0000EAF720958091EE0282230E945D0D0895F0
:101B100021E030E001C0220F8A95EAF78091EE02C1
:101B200082270E945D0D08959091EE02892B0E94FC
:101B30005D0D08959091EE0289230E945D0D089538
:101B40009091EE0289270E945D0D08950895962FC9
:101B50009770A1E001C0AA0F9A95EAF793E07695F5
:101B600067959A95E1F7FB01EE0FFF1F6E0F7F1F40
:101B7000FA01E60FF71F40E050E0682F70E0908117
:101B80009B01042E02C0369527950A94E2F7217036
:101B9000219529272A23292721934F5F5F4F43301F
:101BA000510569F708959B01782F777043E096956A
:101BB00087954A95E1F7FC01EE0FFF1F8E0F9F1FDF
:101BC000F901E80FF91F40E050E080E0219130E09A
:101BD000072E02C0369527950A94E2F72170332725
:101BE000042E01C0220F0A94EAF7822B4F5F5F4F49
:101BF0004330510559F70895282F953070F48F30F0
:101C000060F4862F622F70E02FE0929F600D711DAF
:101C1000112440ED52E00E94A70D0895953070F414
:101C20008F3060F4292F90E060ED72E03FE0239F59
:101C3000800D911D11240E94D30D089580E0089518
:101C4000CF92DF92FF920F931F93CF93DF936C019C
:101C50000091EE028091EF02082BC7E0D0E010E087
:101C6000C8010C2E02C0959587950A94E2F780FD75
:101C700004C02197A8F7F12C07C0FC2EB6018C2FC9
:101C80000E94FD140197A9F38F2DDF91CF911F9131
:101C90000F91FF90DF90CF900895CF93DF93EC01E9
:101CA0000E94200EBE010E94FD14DF91CF91089585
:101CB0001F93CF93DF93EB019091CF02992321F0F3
:101CC000CB010E944D0E13C0882349F0CB010E9426
:101CD000200E182F682FCE010E94FC0D04C0CB01EE
:101CE0000E940E0E182FBE01812F0E94FD14DF915D
:101CF000CF911F9108951F93CF93DF93C091F0026E
:101D000016E08091F102C81799F0D0E01C9FF00115
:101D10001D9FF00D1124EE50FD4F408151816281D5
:101D20007381848195810E942E0D2196C770E9CF21
:101D3000DF91CF911F910895409122035091230389
:101D400060912403709125038091260390912703CD
:101D50000E942E0D08950F931F93CF93DF938091D0
:101D6000270382958F7009F05AC08091240388233D
:101D700009F455C08091F0021091F10260912203A4
:101D800070912303C0912503D091260391E06F3F0A
:101D900009F090E0292F06E0811709F440C0209750
:101DA00021F07F3F21F030E003C031E001C0322F4D
:101DB00090E030FD31C0089FF001099FF00D112423
:101DC000DF01AE50BD4F11963C911197371324C0DF
:101DD0003C91361321C012963C91129731111CC0D0
:101DE00013964D915C9114974C1B5D0B483C51052B
:101DF00098F4809127038F70806180932703E950C6
:101E0000FD4F80818F708061808382E293E00E9429
:101E10009E0C0E947B0E03C001968770BDCFDF91A0
:101E2000CF911F910F910895A1E1B0E0EAE1FFE0A9
:101E30000C94C82D8C0185E0F801DE011D960190FF
:101E40000D928A95E1F7F801E2809091220360916A
:101E5000230320912503309126032115310531F00C
:101E60006F3F31F481E09F3F19F403C081E001C06E
:101E700080E0F82FF1709F2E80FD40C1F801408175
:101E80005181A380B48082E2C82E83E0D82EF090E6
:101E90002403F501E21BF30BFF2009F4DAC0809163
:101EA0002703E83CF10508F096C0282F207F09F0B1
:101EB00053C0561313C0491311C0FE2CE1100EC0BD
:101EC0008F708061809327030E949C0EC6010E9440
:101ED0009E0C80912703F80185834DC1A114B104A4
:101EE00031F05F3F31F481E04F3F19F403C081E0EE
:101EF00001C080E080FD03C081E08E2502C080E04B
:101F000090E0F82FF170FF2E80FF1CC08091F0024E
:101F10002091F10236E0821709F40BC190E0389F5E
:101F2000F001399FF00D1124EE50FD4F61815613E1
:101F300006C06081461303C06281E61203C00196A9
:101F40008770E9CFFE2CEE2009F415C1809127039C
:101F500081608093270354C0561306C0491304C000
:101F6000E11002C0F80199C0C8010E94090D882340
:101F700061F1EE2051F120912703822F82958F701D
:101F800090E0029774F08091220390912303988748
:101F90008F831986BB86AA862C87CE0107960E945E
:101FA0009E0C86E0F801A2E2B3E001900D928A95C2
:101FB000E1F70E94AB0E0E949C0E0AC0561711F169
:101FC000C8010E94090D81112CC0C8010E949E0CFD
:101FD000FF24F394D0C0282F207F81F77A2DB98A6F
:101FE000A88A6E2D89890E94240D82E293E00E94C6
:101FF0009E0C86E0F60111928A95E9F70E949C0EEC
:10200000F12CB9C04913DCCFE110DACFF801858398
:10201000C8010E949E0C86E0F60111928A95E9F7AC
:10202000AAC0EE2091F220912703822F82958F7013
:1020300090E002970CF4B5CF809122039091230396
:102040009A8389831B82BD82AC822E83CE01019646
:10205000A6CFE83CF10508F044C0FE2CEE2009F4C0
:10206000B4CF561330C049132EC02091270320FD52
:1020700021C0822F82958F70482F50E04115510565
:10208000C9F0F80125834F30510541F08F5F982F3B
:102090009295907F822F8F70892B8583C8010E9433
:1020A0009E0C86E0F801A2E2B3E001900D928A95C1
:1020B000E1F73CC086E0F801A2E2B3E001900D92A6
:1020C0008A95E1F758C0C8010E94090D811169CFB6
:1020D00080912703816080932703C8010E949E0C92
:1020E0004AC07A2DB98AA88A6E2D89890E94240D4A
:1020F00086E0F60111928A95E9F718C0EE2009F4FE
:1021000064CFC8010E94090DF82E882309F45DCF21
:1021100086E0F801A2E2B3E001900D928A95E1F722
:1021200082E293E00E9439090E94AB0E0E949C0E4D
:1021300022C04D875E878D859E850E944D0E292F7A
:1021400022952F70223028F49F7039F0811105C03C
:102150000BC0243028F49F7049F4805E883020F052
:10216000C8010E949E0C9F2CF92C05C0F801958196
:10217000907F99F7F9CF8F2D6196EBE00C94E42DC9
:10218000ACE0B0E0E6ECF0E10C94D02D4F83588742
:1021900069877A878B879C87CE0107960E94140FE8
:1021A0008823D1F09F8188852A853B85232B31F0B8
:1021B0008F3F31F481E09F3F19F403C081E001C0FB
:1021C00080E080FD47C04F81588569857A858B8581
:1021D0009C850E942E0D3EC086E0FE013796DE01F2
:1021E000119601900D928A95E1F7FF81E8856A8545
:1021F0007B856115710531F0EF3F31F481E0FF3FE0
:1022000019F403C081E001C080E080FD23C020916B
:10221000F10230E0C9010196877099274091F002E0
:1022200050E084179507F1F1F983EA837D836C838D
:1022300096E0929FD001939FB00D1124AE50BD4FF8
:10224000FE01319601900D929A95E1F78093F1028B
:102250000E947B0E16E08091F0029091F1028917A6
:1022600071F1189FC00111248E509D4F0E94140FD0
:10227000882329F1E091F0021E9FF0011124EE5015
:10228000FD4F4081518162817381848195810E94DB
:102290002E0D8091F00290E001968770992780932F
:1022A000F002D9CF0E94E90C1092F1021092F002D4
:1022B000E2E2F3E086E0DF011D928A95E9F72C96D1
:1022C000E3E00C94EC2D8091300385958595859500
:1022D000089580913003877008959091300397702E
:1022E00081E009F480E0089580913B030895909186
:1022F0003B03892B80933B030895809590913B038A
:10230000892380933B03089510923B030895909195
:102310003A03892B80933A030895809590913A036C
:10232000892380933A03089510923A030895809187
:102330003103089508950E949A1108950E949B11F7
:1023400008959091810392FF08C0909131039817EE
:1023500021F0809331030E949E11089580913103F2
:10236000882329F01092310380E00E949E11089585
:10237000CF93DF93E0910001F091010180913B0345
:102380008083E0910001F0910101908180913A03F6
:10239000892B808380913103882381F0E0910001B3
:1023A000F09101019081892B8083809100019091AF
:1023B00001010E94522481110E94AE11C0910001BE
:1023C000D091010148E050E068E273E0CE010E9444
:1023D0000C2E892B59F088E0FE01A8E2B3E00190B1
:1023E0000D928A95E1F7CE010E94B923DF91CF913A
:1023F00008950E949A1108959091810392FF11C04F
:1024000098E0899F90011124262B209330030E948D
:102410006F0D809130038595859585950E94F91102
:1024200008950E946F0D08951092300380E00E947D
:10243000F911089520913003809582238093300311
:10244000982F977099F430E0482F082E000C550B08
:102450002417350759F09091810392FF07C08595A5
:10246000859585950E947B0D0E9414120895CF9347
:102470009091810392FB222720F92817F9F0C82FA9
:10248000892FC0FB82F98093810380918003909112
:1024900081030E94941282E00E941A1280915003DC
:1024A00080FF0CC01F92CF938DED93E09F938F938D
:1024B0000E9437070F900F900F900F90CF910895C3
:1024C0008091810382FB882780F991E089270E940F
:1024D0003712089581E00E943712089580E00E942B
:1024E000371208956FEF7FEF80E090E00E944E2E4C
:1024F000089580E090E00E942A2E873E9E4F19F4B6
:102500000E94C91A089580E0089582E090E00E9438
:10251000222E089583E090E00E94222E089584E008
:1025200090E00E942A2E0895BC0184E090E00E9471
:102530004E2E0895AB01BC018FE090E00E94422E28
:102540000895AB01BC0183E190E00E94422E089502
:1025500060E070E0CB010E94A112089560E070E09D
:10256000CB010E949A120E94A812089567EE7EEF96
:1025700080E090E00E944E2E60E082E090E00E94B9
:10258000302E60E083E090E00E94302E1092EF0247
:1025900060E074E184E090E00E944E2E60E086E00E
:1025A00090E00E94302E6FEF87E090E00E94302E86
:1025B00040E050E0BA0188E090E00E94422E60E0E6
:1025C0008DE090E00E94302E40E050E0BA0188E1BA
:1025D00090E00E94422E60E087E190E00E94302E61
:1025E00040E050E0BA018CE190E00E94422E60E0B1
:1025F00070E080E290E00E944E2E40E050E0BA0190
:1026000088E190E00E94422E80E00E94E21A0E943F
:10261000171B0E94AE1208950E94B6120895682FEB
:102620008EE090E00E94302E08950E946525609310
:102630004C0370934D0380934E0390934F0360932C
:1026400048037093490380934A0390934B03089582
:1026500081E008950E942813089508950E942D1383
:1026600008950E942D1308950E94311308950E9429
:102670002D1308950E94371308950E942D13089575
:1026800086E797E20E94A2230E943D130E943A131C
:1026900008950E942E130E942D1308950E94FB1589
:1026A0000E94AA0808950E9450250E94271B0E949C
:1026B00014170E944E130E9434130895AAE0B0E04C
:1026C000E4E6F3E10C94C62D0E942A172EE3E22ED5
:1026D00023E0F22E5701D12CF501019111915F01F8
:1026E0008D2D0E94161680279127D394F5E0DF16D2
:1026F00019F0892B89F322C0892B01F50E945925F5
:102700008C0180913C0390913D030817190709F44F
:102710005BC08FEF89838A831B820E945925816069
:10272000782F9D838C8349815A816B818D810E9492
:10273000F80810933D0300933C0346C0809150037A
:1027400081FD0E941F160E942A13782E10E0812F0F
:102750000E9416164C01F701A080B180A826B92668
:10276000A114B10449F100E0CC24C394D12CC501DB
:102770008C219D21892BC1F07720B1F00E831F831E
:1027800021E0C4018C219D21892B09F420E02887B8
:102790000E9459258160782F9A8789874E815F81B1
:1027A00068858A850E94F8080F5FCC0CDD1C0F300D
:1027B000F1F6F701918280821F5FF2E0EF0EF11CCB
:1027C000153029F60E9415130E94C9190E94BD08F0
:1027D0002A96EDE00C94E22DCF93DF930E94021530
:1027E000EC01811520E59207E0F5811530E49307AF
:1027F00008F09FC0803E910528F58D3C910508F0BA
:1028000096C0883A910570F4853A910508F085C024
:102810008130910509F47EC008F4DCC0049708F00B
:10282000DCC0D8C0813C910508F0D4C0C85AD0E0C3
:10283000CC0FDD1FC85BDE4F0990D881C02DCE01C3
:102840009464CCC0811540E2940708F0B8C08115AB
:1028500051E0950708F0C1C0883E910508F4BDC05D
:10286000B9C0803662E5960720F5803472E5970797
:1028700008F06CC0C03282E5D80708F05EC0C11510
:1028800092E5D90708F489C02C2F2695269560E299
:10289000269F90011124C37081E090E002C0880F50
:1028A000991FCA95E2F7E901C82BD92BCE019D6883
:1028B00095C0803A22E59207E0F48F71C03832E586
:1028C000D30708F059C08695869570E2879F9001DE
:1028D00011249C2F9370C1E0D0E0AE0102C0440FE0
:1028E000551F9A95E2F7EA01DA68C9018C2B9D2BF6
:1028F00075C0803C42E5940708F445C0803E92458F
:1029000008F068C0CF71DD27DC2FCC27CE01806FA7
:10291000906A64C081E090E061C0C55AD0E0C658BA
:10292000DE4F8881C82FD0E0CE01906457C09065FB
:1029300055C0DF70CE01906A51C0CF718C2F90E0EE
:10294000D82FCC27CE01816F906A48C08F718695B1
:10295000869570E2879FA00111249C2F937021E03F
:1029600030E0B90102C0660F771F9A95E2F7CB01FC
:102970009C68842B952B32C090E0D82FCC27CE01B9
:10298000846F906A2BC08F710E949E158F7190E0AA
:10299000D82FCC27CE01906221C08C2F8F710E943E
:1029A0009E1595E0D695C7959A95E1F7CF70D0E042
:1029B000DC2FCC27D069BE01682BCB010FC08D2F37
:1029C0008F710E949E15DD27D0628F719E01382B7A
:1029D000C90104C080E090E001C0CE01DF91CF9139
:1029E0000895753038F46F3028F4462F672F0E9411
:1029F000DD21089580E090E008950E94F1140E9486
:102A0000EC1308958238910569F1B0F48133910592
:102A100009F475C048F48932910509F467C08A3217
:102A2000910509F471C008958533910509F459C0E1
:102A300089339105B9F00895833E910589F138F401
:102A4000803E9105D1F0823E910529F10895863EA0
:102A50009105C9F1873E9105D9F1843E910509F0B0
:102A60006CC027C02091800320FD57C021FD55C0B8
:102A70002091810323FD5BC008958091800380FD38
:102A800048C08091810380FF48C08091800384FD0D
:102A900046C083EE51C08091800382FF3CC0F5CFD9
:102AA0008091800382FD37C08091810380FD35C015
:102AB000ECCF8091810381FF36C08091800384FD3B
:102AC0002EC087EE39C08091800383FF2AC0F5CFE6
:102AD0008091800383FD25C08091810381FD23C007
:102AE000ECCF8091800385FD22C01FC080918003C0
:102AF00085FD1BC08091810383FF19C00AC08091AE
:102B0000800386FD16C017C08091800386FD13C028
:102B100010C089E311C082EE0FC080EE0DC080E0CE
:102B20000BC086EE09C084EE07C085E305C089E2CC
:102B300003C08AE201C081E390E008959091800390
:102B400092FF0DC0282F2871283019F4877F8460E8
:102B500006C0282F2471243011F48B7F886093FFE6
:102B60000DC0282F2871283119F4877E846106C092
:102B7000282F2471243111F48B7E886120918103E8
:102B800020FF0DC0382F3871383019F4877F8160ED
:102B900006C0382F3171313011F48E7F886021FFEB
:102BA0000DC0282F2871283119F4877E816106C055
:102BB000282F2171213111F48E7E886194FD877E4A
:102BC00008950E94721208950E942A178FE39CE9CB
:102BD0000197F1F700C000000E942A1780E00E94D0
:102BE000161680FF04C00E94E1150E94A6250895D4
:102BF0000E94E41508950E947912811102C00E947A
:102C00000C130E948512809350030E948F129093A0
:102C10008103809380030E94F8150E948A120E940B
:102C2000450D8091EE020E945A0D0895E82FF0E0C4
:102C3000EE0FFF1FE457FC4F808191810895A0E0C3
:102C4000B0E0E5E2F6E10C94CB2D82E094E00E9446
:102C50009E068CE8E82E83E0F82EC0E0D0E09DEFE1
:102C6000C92E93E0D92E04EF13E0DF93CF93DF92C8
:102C7000CF920E9437078AEF93E00E949E06F701E9
:102C8000819191917F010E9481089F938F931F935F
:102C90000F930E94370782EF93E00E949E062196D1
:102CA0008DB79EB708960FB6F8949EBF0FBE8DBF26
:102CB000C530D105D1F6CDB7DEB7E8E00C94E72DED
:102CC00080EA8A95F1F7089500C008950E94601681
:102CD000089508950E94691608950E946A1608953D
:102CE0000E94691608950E9470160895F894E82FBE
:102CF000E295EF70F0E031A1282F2F7081E090E095
:102D000001C0880F2A95EAF7982F9095932391A3F5
:102D100092A1892B82A3789408950F931F93CF9348
:102D2000DF93CCE8D1E089918F3F11F00E947616B5
:102D300081E0C139D807B9F7CDE7D1E00CE811E05F
:102D400089918F3F11F00E9476160C171D07C1F76D
:102D5000DF91CF911F910F910895A0E0B0E0E3EBD8
:102D6000F6E10C94CA2D8C01C62FD0E0CE01845719
:102D70009E4F6C01FC0190819F3F09F450C0B62E1C
:102D8000F894E92FE295EF70F0E081A19F7021E0C7
:102D900030E001C0220F9A95EAF7822B81A382A12D
:102DA0002095282322A378940E946416EDE7F1E091
:102DB0004CE851E021E030E0E12CF12C61916F3FD3
:102DC00089F0A62FA295AF70B0E090968C9190E01C
:102DD0006F7002C0959587956A95E2F780FD02C0F5
:102DE000C90102C080E090E0E82AF92A220F331FCF
:102DF0004E175F0719F7F60180818F3F11F00E948F
:102E0000761661E0E114F10409F460E08B2D0E9474
:102E10006616CC0FDD1FC00FD11FF982E882CDB737
:102E2000DEB7E9E00C94E62D0E948D168AE0ECE80E
:102E3000F3E0DF01982F1D929A95E9F7E2E8F3E0BD
:102E4000DF011D928A95E9F785E00E9465170E94CF
:102E5000D4070895AAE0B0E0E0E3F7E10C94CE2DAA
:102E60008E010F5F1F4F8AE0F80111928A95E9F7F2
:102E7000F12C6F2DC8010E94AD16F394F5E0FF12FE
:102E8000F8CF4AE050E0B80182E893E00E940C2EAF
:102E900021E0009709F420E0892B41F08AE0F80155
:102EA000A2E8B3E001900D928A95E1F745E06CE865
:102EB00073E082E893E00E946617182F0E94D707FC
:102EC000812F2A96E5E00C94EA2D0895EF92FF9267
:102ED0000F931F93CF93DF937C018B01C42F222389
:102EE00049F081E0809353030E9459259093520347
:102EF0008093510380915303811102C080E01CC074
:102F000080915103909152030E9471250597B0F36F
:102F1000D0E0CC0FDD1FAE01B701C8010E940C2E1E
:102F2000892B39F0AE01B701C8010E94192E81E04A
:102F300001C080E010925303CDB7DEB7E6E00C94F9
:102F4000E92D0E94F3270E9453130E940028089540
:102F50000E9405280E945E130E94232808950E9463
:102F6000F0240E94D9270E9440130E94A1170E94BA
:102F7000A8170E944913FBCF80915A0380FF06C017
:102F80006091070170E0660F771F26C081FF04C0C3
:102F90006091070184E005C082FF07C060910701CE
:102FA00088E0689FB001112417C0909159039923BC
:102FB000D1F060910601961788F72091070188E00B
:102FC000289F90011124929FA001939F500D1124DE
:102FD00070E0CA010E94A02D6038710540F46115AF
:102FE000710519F406C068E070E0862F08958FE738
:102FF000089581E0089580915A0380FF08C0609190
:10300000030170E0759567957595679521C081FFFF
:1030100006C06091030170E07595679519C082FF45
:1030200004C06091030170E010C09091580399238F
:1030300099F0609102019617A0F780910301899F92
:10304000C001112470E00E94A02D6038710540F489
:103050006115710519F406C061E070E0862F0895CE
:103060008FE7089581E008958D3C21F40E94BC17FC
:10307000819504C08E3C29F40E94BC1780935E03A6
:1030800008958F3C21F40E94BC17819504C0803DB7
:1030900029F40E94BC1780935D030895893D19F4BB
:1030A0000E94FB1705C08A3D31F40E94FB178195F1
:1030B00080935F0308958B3D21F40E94FB17819557
:1030C00004C08C3D29F40E94FB178093600308958F
:1030D0009FE2980F983078F421E030E0A90102C017
:1030E000440F551F9A95E2F7CA0190915C03892B12
:1030F00080935C0308958D3D21F480915A03816093
:103100000BC08E3D21F480915A03826005C08F3D33
:1031100029F480915A03846080935A0308958D3C6A
:1031200039F490915E0397FF35C010925E0359C049
:103130008E3C29F490915E031916BCF32BC090913C
:103140005D038F3C29F497FF25C010925D0349C0B1
:10315000803D19F41916CCF31DC090915F03893D91
:1031600029F41916BCF410925F033BC08A3D19F490
:1031700097FF10C0F8CF8B3D39F49091600397FF13
:1031800009C0109260032DC08C3D21F49091600322
:103190001916BCF39FE2980F983080F421E030E0DC
:1031A000A90102C0440F551F9A95E2F7CA01809504
:1031B00090915C03892380935C0313C08D3D21F4BF
:1031C00080915A038E7F0BC08E3D21F480915A036B
:1031D0008D7F05C08F3D29F480915A038B7F8093AA
:1031E0005A0380915D03811106C080915E038111B5
:1031F00002C01092590380915F03811106C0809133
:103200006003811102C01092580308958091500309
:1032100083FF7EC080E494E00E949E0680915C0360
:103220001F928F938BE394E09F938F930E943707B5
:1032300089E394E00E949E0680915D03282F082E6A
:10324000000C330B3F938F9386E394E09F938F930F
:103250000E94370784E394E00E949E0680915E03FB
:10326000282F082E000C330B3F938F9381E394E0BB
:103270009F938F930E9437078FE294E00E949E06EF
:1032800080915F03282F082E000C330B3F938F9300
:103290008CE294E09F938F930E9437078AE294E038
:1032A0000E949E0680916003282F082E000C330B8D
:1032B0003F938F9387E294E09F938F930E94370709
:1032C00084E294E00E949E06809159031F928F939E
:1032D00081E294E09F938F930E9437078FE194E0FF
:1032E0000E949E0680915A031F928F938CE194E076
:1032F0009F938F930E94370789E194E00E949E0676
:103300008DB79EB74C960FB6F8949EBF0FBE8DBF7B
:103310000E94592520915D03211104C020915E0374
:10332000222321F0909357038093560320915F034B
:10333000211104C020916003222321F090935503B2
:10334000809354038BE593E00E94FA230895EBE504
:10335000F3E086E0DF011D928A95E9F710925903A8
:103360001092580310925A030895FC018281811132
:103370000DC0838181110AC08481811107C091E051
:103380008581811101C090E0892F01C081E08170A9
:103390000895A6E0B0E0EFECF9E10C94D02D86E0C2
:1033A000EBE5F3E0DE01119601900D928A95E1F7CD
:1033B00010925D0310925E0310925F0310926003FF
:1033C0008B81811104C08C81882309F45FC08091B6
:1033D0005603909157030E947125AC0190915903B7
:1033E000992339F02091080130E02417350758F06F
:1033F0004DC0209109018AE0289F900111242417D3
:10340000350718F043C09F3F19F09F5F9093590311
:103410001B81112361F00E94BC17111614F09FEF5D
:1034200001C091E0989F902D112490935D031C8121
:10343000112361F00E94BC17111614F09FEF01C018
:1034400091E0989F902D112490935E0330915D033D
:103450003323E1F020915E032223C1F045EB3403D6
:10346000C0011124992319F090935D0303C081E0FA
:1034700080935D0335EB2303C0011124992319F0D8
:1034800090935E0303C081E080935E038D81811180
:1034900004C08E81882309F45FC080915403909109
:1034A00055030E947125AC0190915803992339F07E
:1034B0002091040130E02417350758F04DC02091C9
:1034C00005018AE0289F900111242417350718F080
:1034D00043C09F3F19F09F5F909358031D811123B4
:1034E00061F00E94FB17111614F09FEF01C091E0EC
:1034F000989F902D112490935F031E81112361F0FA
:103500000E94FB17111614F09FEF01C091E0989FE5
:10351000902D11249093600330915F033323E1F0E9
:10352000209160032223C1F045EB3403C001112434
:10353000992319F090935F0303C081E080935F03A8
:1035400035EB2303C0011124992319F090936003F4
:1035500003C081E080936003BE016F5F7F4F8BE506
:1035600093E00E94A124811105C08BE593E00E94A5
:10357000B51981110E94061986E0FE013196ABE56E
:10358000B3E001900D928A95E1F72696E3E00C9462
:10359000EC2D82E290E00E94222E823281F483E2BE
:1035A00090E00E94222E823151F484E290E00E9449
:1035B000222E91E0883009F090E0892F01C080E050
:1035C00081700895CF93C82F811102C06FEF01C0A1
:1035D00062E282E290E00E94302EC11102C06FEFE1
:1035E00001C062E183E290E00E94302EC11102C06E
:1035F0006FEF01C068E084E290E00E94302ECF912E
:103600000895089585E290E00E94222E682F70E0D0
:1036100080E090E008950895CF93C62F0E940B1B81
:103620006C2F85E290E00E94302ECF91089580E0CB
:103630000E94E21A60E070E0CB010E940C1B0E9425
:1036400070210E94322281E00E94E21A08950E94B5
:10365000011B0E94021B0E940B1B0E94C91A8111B0
:1036600002C00E94171B08950895CF93FB01C281E9
:10367000CC23E9F09C01225037472031310520F45A
:1036800082500E9442220CC08115F7E79F0751F437
:1036900081E00E946F0D43E062E081E00E94CA0772
:1036A000C0E018C081309747A9F482E0F2CF8115BD
:1036B000E7E79E0711F481E004C08130974749F4A1
:1036C00082E00E947B0D43E062E081E00E94CA0735
:1036D00001C0C1E08C2FCF9108952FEFFC01208312
:1036E00008950E946D1B089580E00895EF92FF9267
:1036F0000F931F93CF93DF93EC01062F0E94741B4F
:103700008111B1C0E8818E2F90E0FC013197E33147
:10371000F10508F0A2C0EE59FF4F0C94B42D1982A8
:103720008BE05EC08981823089F030F4813009F00D
:1037300094C00E9465250CC0833079F0843009F074
:103740008CC01A821B821C821D8289C00E94021BAF
:103750009A838B837C836D8382C07E0110E0812FEE
:103760000E941616F701928383831F5FF2E0EF0E2B
:10377000F11C1530A1F773C08981823039F0853092
:1037800009F06BC08A810E94341B69C06A817B8109
:103790008C819D810E94BA2D0E940C1B60C04B81C0
:1037A0006A8189810E9434219C838D8358C02C8139
:1037B0003D813227232732274B816A8189810E94EC
:1037C00055214DC00E9470214AC0602FCE010E9439
:1037D000711B45C00E94E92124C00E94EB219983FE
:1037E0008A833DC06B8170E089819A81AE014C5F14
:1037F0005F4F9827892798270E94EE2130C06B8160
:1038000070E089819A81AE014C5F5F4F98278927CC
:1038100098270E94112223C00E94322220C00E94B9
:10382000212189831CC06B8170E089819A81AE015E
:103830004C5F5F4F9827892798270E949B210FC0D4
:103840006B8170E089819A81AE014C5F5F4F982750
:10385000892798270E94BD2102C08FEF8883602F9F
:10386000CE010E940B26CDB7DEB7E6E00C94E92D21
:10387000CF93DF93FC01DB0112968C91882309F42E
:10388000DDC09F0130572332310508F0D8C0EF0169
:103890000E948F129093810380938003FE01E15078
:1038A000F047E232F10520F4EB58FF4F0C94B42DB1
:1038B000809180038160AAC0809181038860B2C03A
:1038C000809180038260A2C08091800320C080919B
:1038D000800388609BC0809181031EC0809181031A
:1038E0008260A0C080918003806190C0809180033D
:1038F00080628CC080918003806488C00E94E90C43
:1039000080918003806882C0809180038860846099
:103910007DC0809181038260816084C0809180033A
:103920008E7F74C080918103877F7CC080918003EB
:103930008D7F6CC08091800320C080918003877F41
:1039400065C0809181031EC0809181038D7F6AC014
:10395000809180038F7E5AC0809180038F7D56C0F6
:10396000809180038F7B52C00E94E90C809180037C
:103970008F774CC080918003877F8B7F47C0809179
:1039800081038D7F8E7F4EC08091800382FB222732
:1039900020F991E0922790FB82F990FB83F936C0E1
:1039A00080918103982F909591708E7F892B90FB49
:1039B00081F938C08091800386FB222720F991E0AD
:1039C000922790FB86F922C00E94E90C8091800327
:1039D00087FB222720F991E0922790FB87F916C0F8
:1039E00081E001C080E00E940F131EC0809180031F
:1039F00084FB222720F991E0922790FB84F906C0EE
:103A000080918003982F909590FB80F9809380039C
:103A10000BC08091810383FB222720F991E092273C
:103A200090FB83F9809381038091800390918103BF
:103A30000E9494120E94E90C80E001C081E0DF91B5
:103A4000CF910895A0E0B0E0E8E2FDE10C94CC2D28
:103A5000E82FF0E0ED59FB4FD490282F26952695BE
:103A6000269530E0F901ED5FFA4F0491877010E080
:103A7000082E02C0159507950A94E2F701701127E8
:103A8000F901ED50FB4FE490F12C082E02C0F594A3
:103A9000E7940A94E2F791E0E922FF24F901ED515D
:103AA000FB4FC491D0E002C0D595C7958A95E2F747
:103AB000C170DD270115110519F081EE0E94490939
:103AC000E114F10419F086EE0E9449098D2D0E943F
:103AD0007C0AE114F10419F086EE0E94F809011540
:103AE000110519F081EE0E94F809CD2B19F08CE236
:103AF0000E947C0ACDB7DEB7E7E00C94E82DEF9288
:103B0000FF920F931F93CF93DF93EC01162F0AE0E0
:103B10008881882309F455C0813009F043C0898128
:103B2000813041F47E0182E0E80EF11C8A810E941E
:103B30007C0A09C0823049F47E01E2E0EE0EF11CFD
:103B40008A810E944909E7012FC0833041F47E0138
:103B5000F2E0EF0EF11C8A810E94F809F4CF843064
:103B600011F0219621C02A81229680E090E030E079
:103B7000205331092A30310558F4089FA001099FCC
:103B8000500D1124C901840F951F21962881EFCF74
:103B9000009751F0EFE9FFE03197F1F700C0000026
:103BA0000197F6CF0E94221D2196812F882309F4C8
:103BB000AFCFEFE9FFE03197F1F700C0000081508F
:103BC000F5CFCDB7DEB7E6E00C94E92D8091020188
:103BD0001F928F93809103011F928F938091060112
:103BE0001F928F93809107011F928F9380910801FC
:103BF0001F928F93809109011F928F9383E195E02B
:103C00009F938F930E9437078DB79EB70E960FB67E
:103C1000F8949EBF0FBE8DBF0895883220F58E3177
:103C200008F068C08B3091F1C0F4873009F0BEC055
:103C300081E08093090184E1809308018AE0809308
:103C400007018EE18093060188E08093030188E2FA
:103C50008093020185E796E0C6C0833109F443C032
:103C6000843169F1A3C08F3409F49EC028F48932ED
:103C700031F1883359F09AC0813531F008F4D4C05D
:103C8000823509F4A7C092C08FEFA5C087E996E0FE
:103C90000E949E060E94E61D1F9281E08F931F9254
:103CA00088E08F9380E995E09F938F930E94370778
:103CB0000F900F900F900F900F900F9096C084E987
:103CC00096E00E949E0680916503882309F4AAC0AD
:103CD00010926503109264031092630310926203C2
:103CE00010926103B1C086E896E00E949E060E9491
:103CF000E61D7BC08D5180936503833031F170F4F4
:103D00008130D1F0823009F03FC088E091E090939B
:103D10006403809363038EE991E01FC0853059F1FD
:103D200008F1863089F582E091E0909364038093F6
:103D3000630389ED91E011C089E091E09093640301
:103D40008093630385E991E008C087E091E0909358
:103D50006403809363038AEA91E090936203809303
:103D6000610318C086E091E090936403809363033D
:103D700087EB91E0F2CF83E091E09093640380932E
:103D8000630386EC91E0E9CF1092650383E896E047
:103D90000E949E0680916503882309F455C01F92F6
:103DA0008F938FE796E00DC08AE015C082E796E01A
:103DB0001AC097FF47C0108280811F928F938CE6B4
:103DC00096E09F938F930E9437070F900F900F906C
:103DD0000F900BC081E0E0916303F0916403309792
:103DE00029F589E696E00E949E062091650322232C
:103DF00059F18091610390916203009711F481E978
:103E000091E09F938F931F922F9380E696E09F936C
:103E10008F930E9437070F900F900F900F900F9085
:103E20000F9016C080E0089586EFD5CF2081082E30
:103E3000000C990B820F911D8F3F910509F00CF436
:103E4000B8CF8FEF8083B8CF8CE596E00E949E06B6
:103E500081E00895CF93C82F1F928F938DEA96E04B
:103E60009F938F930E94370781E001C0880FCA9506
:103E7000EAF70E94450D0E94E90C0F900F900F90F9
